:020000040000FA
:040000000000C6280E
:040004000034003490
:080008008B13F000030E8301CD
:10001000F2000A08F1008A018C1811288C1A552860
:1000200046288C105118BF285308031D282806089D
:100030006502031D252805080F39D600D60E0708CE
:100040000F39560766020319BF280A30D300BF28AC
:10005000D30BBF280608650203193B280608E500F4
:1000600005080F39E600E60E07080F39E607501CB1
:10007000BF285114BF2805080F39D600D60E07082F
:100080000F3956076602031D3028BF28D40B4D28B0
:1000900083160C128312D401BF28051E4828D50AE6
:1000A0005508840000089900BF281A08BC008C126B
:1000B0003B18B028BA1B8328300884003108840715
:1000C00000083C02031D6E28B10A05303102031DF1
:1000D0006F28B101B901FF30BA00BF28B10138085B
:1000E00084003908840700083C02031D8128B90AEE
:1000F00005303902031DBF28B101B901FF30BA0034
:10010000BF28B901BF283C08BA00FF30BB0000304F
:100110008A003A080F399A20CD004D080319982813
:10012000BD01CE01CD1FBF28CD132808CE00BF28AA
:10013000D217BF28D70000308A0057080F3982072E
:10014000003400348034013400340034003400348E
:1001500000340534013400340034003400340034F9
:10016000CE080319B528CE03BF28400884003D08F7
:1001700084073C088000BD0ACD0BBF28D217710848
:100180008A00720E8300F00E700E090083120313B2
:100190004130C000BD01C101C201C301C401C5019C
:1001A000C601C701C801D001D101D3012030B80078
:1001B00083120313B9013808840039088407031730
:1001C0008D0083160C1483120C0803138000B90AE7
:1001D0000F303902031DDB285330B2005730B30013
:1001E0004E30B4003030B5003030B6003230B000A0
:1001F000B1012930B800BA01BB01BD01D20183129F
:1002000003138501831606309F00DF308500FF3021
:100210008600AF308700831283160330920083126A
:100220007D3092008316203099002430980083128C
:10023000903098008B170B1783168C148C16831232
:10024000D21B4529511825292029D118382985166E
:10025000051E202907160D30D4006030D50084001B
:1002600000089900831603130C168312D114202959
:10027000D408031D20298316981C432983120712D2
:100280008512D101202983122029BD01BB01013033
:100290008A003A080F394F3E03188A0A8200C6289E
:1002A0006229622966295F295F295F295F295F2901
:1002B0006B295F295F295F295F295F295F29BA01BF
:1002C000D20120295114BA01D20120294108D000BD
:1002D000BA01D20120294108A9004208AA00430816
:1002E000AB004408AC004508AD000930D800293007
:1002F000D9000530BE00BA01D2018B135908840021
:10030000000803178C000313580803178D00831689
:100310008C110C1555308D00AA308D008C140C11E9
:10032000031383120D1E92290D12D80AD90ABE0B8F
:0C0330007D29B901BA01BB018B172029FF
:02400E00323F3F
:1042000000000000000000000000000000000000AE
:104210000000530057004E003000300020005300D3
:104220005700310036002000560031002E003000CB
:04423000300030002A
:00000001FF
